:020000040000FA
:060000004AEF10F01200AF
:0600080004EF04F01200F9
:060018000CEF04F01200E1
:060800004AEF10F01200A7
:0608080019EF0DF01200D3
:0608180020EF0DF01200BC
:06082A000100B2200000F5
:08083000B60000000300000007
:08083800D9CFE6FFE1CFD9FFA3
:10084000E652A09A6A6A686A706A010EE66EE66A03
:10085000E66A710EE66E0F0EE66E20EC10F00B6E7F
:10086000050EE15E0B50160E6F6E9F0E6B6E7B0ECB
:10087000696EDF6ADF500B6E0C6A080E0B5C000EAF
:100880000C5810E2DF50040DF3CFE9FFF4CFEAFF7C
:10089000000EE926040EEA22EE6AEE6AEE6AEE6ABD
:1008A000DF2AE8D76D8C6E6A6D986D9C68A607D0BC
:1008B00068960001736B786B796B7A6BF7D70001E0
:1008C000010E8A6F8B6F8C6B8D6B806BDF6A020EF3
:1008D000DF5C26E2EA6ADF34FE0BEA36E96E6B0E75
:1008E000E926000EEA22EE6AED6AEA6ADF34FE0BC0
:1008F000EA36E96E670EE926000EEA22EE6AED6A34
:10090000DF50EA6A840FE96E000EEA22EF6ADF50D8
:10091000EA6A860FE96E000EEA22EF6ADF2AD7D76D
:100920000001080E6B6F040E6C6F160E706E0401E2
:10093000200E026F040E036F080E016F840E006F0D
:100940000001616B606BE552E552E7CFD9FF120001
:10095000D9CFE6FFE1CFD9FFE652000160510FE1A8
:100960006D6A696A160E6F6E9F0E6B6E7B0E696EF6
:100970006DB602D06D86FCD70001010E606F600578
:1009800008E16DBA06D0686A696A69806988020EF2
:10099000606F6850040B05E06950040B02E0689436
:1009A000BED86DB24FD06850010B08E06950010B02
:1009B00005E042DF0001040E606F68906850100B84
:1009C00005E06950100B02E095D8689868AC12D029
:1009D00069AC0FD0010EE66EE66A000EE66EE66ABE
:1009E000730EE66EE66A8CEC0EF00B6E060EE15EA0
:1009F0000B50689C6850200B04E06950200B01E00C
:100A000060D86850020B13E06950020B10E0010E31
:100A1000E66EE66A000EE66EE66AE6687F0EE66E51
:100A20008CEC0EF00B6E060EE15E0B506A6A040E43
:100A30000001E76E6019E8AE02D0E73402D0E7505B
:100A4000605D02E2A19A38D069A635D0DF6A040E53
:100A5000DF5C31E268A62FD06CCF81F000018151BC
:100A6000780BE842E842E842826F689681B506D08A
:100A70008251EA6A860FE96E000E05D08251EA6A59
:100A8000840FE96E000EEA22EF70825102E15ED817
:100A900010D0000EE66EE66A810EE66E000EE66E7F
:100AA000720EE66EE66A8CEC0EF00B6E060EE15EE0
:100AB0000B50DF2ACCD7A19AE552E552E7CFD9FFF8
:100AC000120070A015D063C0E9FF64C0EAFFEF50C8
:100AD00080080DE16BC0E9FF6CC0EAFFEF508408AD
:100AE00006E163C0E9FF64C0EAFF8C0EEF6E709010
:100AF000689A1200698468986D820001010E806F07
:100B0000000EE66EE66AE66EE66A750EE66EE66A68
:100B10008CEC0EF00B6E060EE15E0B501200000125
:100B2000806B000EE66EE66AE66EE66A740EE66EAE
:100B3000E66A8CEC0EF00B6E060EE15E0B506D92C9
:100B4000699468A402D06894FCD71200D9CFE6FF5C
:100B5000E1CFD9FFE652FD0E0001811553E17E0E73
:100B60008115E8407F0B040DF3CF63F0F4CF64F000
:100B7000000E6327040E642363C065F064C066F052
:100B8000657563C0E9FF64C0EAFFEF503C0BE842C3
:100B9000E8420D0835E1DF6A080EDF5C23E263C03E
:100BA000E9FF64C0EAFF020EE926000EEA22EE50D9
:100BB000EFCFEAFFE96EEF50E66EDF50EA6A200FF2
:100BC000E96E040EEA22E552E750EF6E63C0E9FFDA
:100BD00064C0EAFF020EE926000EEA22EE2AEF22A6
:100BE000DF2ADAD763C0E9FF64C0EAFF020EE92614
:100BF000000EEA22200EEE6E040EED6E0DD807D028
:100C00003AD805D0FD0E8115040801E159D8E55206
:100C1000E552E7CFD9FF120000016F6B896B8C6B37
:100C20008D6B836B706B6BC0E9FF6CC0EAFFEF9E4E
:100C30006B756BC0E9FF6CC0EAFFEF9E6B7565C01A
:100C4000E9FF66C0EAFFEF9E736B746B756B786BA0
:100C5000796B7A6B8CD8000EE66EE66AE66EE66A11
:100C6000030EE66EE66A8CEC0EF00B6E060EE15E8D
:100C70000B5086EF09F0020E0001705D02E146EFB5
:100C80000AF0706B83511AE165C0E9FF66C0EAFFA4
:100C9000EE52080EEF6E65C0E9FF66C0EAFF020E75
:100CA000E926000EEA22200EEE6E040EED6E65C0FF
:100CB000E9FF66C0EAFF8C0EEF6E1200836B120034
:100CC000D9CFE6FFE1CFD9FFE6526BC0E9FF6CC098
:100CD000EAFFEF50400B01E0010EDF6E00016B7583
:100CE000080E605D08E122C46EFF6E5002E0100E37
:100CF00001D0040E606F700526E16BC0E9FF6CC087
:100D0000EAFF020EE926000EEA22280EEE6E040E1D
:100D1000ED6E5DDB020E00016F5D06E16BC0E9FF69
:100D20006CC0EAFF840E0DD0DF5006E16BC0E9FF16
:100D30006CC0EAFFC80E05D06BC0E9FF6CC0EAFFCB
:100D4000880EEF6E0FD078AF0CD07B517C1107E08E
:100D500005D07CC0FAFF00017B51F96EFADF00017B
:100D6000789F706BE552E552E7CFD9FF120004017E
:100D70002051600BE842E842E842E842E8420009BC
:100D800001E0120021510C0A50E00B0A3FE00C0A6E
:100D900031E0010A22E00B0A1EE0020A1CE0030A0D
:100DA00018E0080A10E0010A0CE00F0A08E0030A44
:100DB00001E012000001738F080E606F1200CFEF88
:100DC00008F0E5EF0AF00001610E716F000E726F1E
:100DD0000CD02CEF09F016EF07F024510001716FD1
:100DE000726B620E7127000E72237381010E746F95
:100DF000738F12000001738F04012451EA6A620F9D
:100E0000E96E000EEA2222C4EFFF1200000EE66E29
:100E1000E66AE66EE66A020EE66EE66A8CEC0EF0B4
:100E20000B6E060EE15E0B5012001200D9CFE6FFEA
:100E3000E1CFD9FF030EE1260401220510E1205184
:100E40001F0B00090CE10001738F030E0401215DEB
:100E500004E10001010E7F6F02D000017F6B0401ED
:100E6000225101E003D120511F0B020801E0FED006
:100E700024510F0B000901E1F9D024510F0B010897
:100E800001E2F4D0200E0001605D01E0EFD0738F2D
:100E9000040124BF16D024510F0BE96EEA6AD890E2
:100EA000E936EA36670EE926000EEA22EECFDEFFCB
:100EB000EDCFDDFF24510F0BEA6A860FE96E000EBD
:100EC00015D024510F0BE96EEA6AD890E936EA365C
:100ED0006B0EE926000EEA22EECFDEFFEDCFDDFF3E
:100EE00024510F0BEA6A840FE96E000EEA22020E0B
:100EF000EFCFDBFFD950020FE96EDACFEAFFEF50F8
:100F0000010B03E1000EDF9401D0DF8424BF0BD07E
:100F100024510F0BE96EEA6AD890E936EA36670E7B
:100F2000E926000E0AD024510F0BE96EEA6AD89028
:100F3000E936EA366B0EE926000EEA22DECFEEFF36
:100F4000DDCFEDFF030E215D20E1DECFE9FFDDCF38
:100F5000EAFFEF50800B11E024BF07D024510F0BA4
:100F6000EA6A860FE96E000E06D024510F0BEA6A7A
:100F7000840FE96E000EEA22EF82840EDECFE9FFD5
:100F8000DDCFEAFFE850EF1271D0DF74DECFE9FF6A
:100F9000DDCFEAFFEF50800B1BE0DECFE9FFDDCFB6
:100FA000EAFFEF9EDECFE9FFDDCFEAFFEF8C020E16
:100FB000E66EE66ADECFE6FFDDCFE6FF050EE66E03
:100FC000E66A8CEC0EF00B6E060EE15E0B5005D05F
:100FD000DECFE9FFDDCFEAFFEF8CDF74D950020FDF
:100FE000E96EDACFEAFFEF50020B0EE1DECFE9FF48
:100FF000DDCFEAFFEF50800B32E0DECFE9FFDDCF3F
:10100000EAFFEF50040B2BE1040124BF07D0245169
:101010000F0BEA6A860FE96E000E06D024510F0B03
:10102000EA6A840FE96E000EEA22EF923B0E0B6E25
:10103000DECFE9FFDDCFEAFFE850EF16020EE66EE5
:10104000E66ADECFE6FFDDCFE6FF050EE66EE66A76
:101050008CEC0EF00B6E060EE15E0B5007D03B0ED3
:10106000DECFE9FFDDCFEAFFE850EF16030EE15CCB
:1010700002E2E16AE552E16EE552E7CFD9FF1200E4
:1010800000018A514DE1010E8A6F8B5149E1010E39
:101090008B6F020E705D0DE16BC0E9FF6CC0EAFF63
:1010A000EE52EF6A6BC0E9FF6CC0EAFFC80EEF6E4C
:1010B0001200700535E1836B63C0E9FF64C0EAFF8D
:1010C000EE52080EEF6E63C0E9FF64C0EAFF020E45
:1010D000E926000EEA22200EEE6E040EED6E63C0CD
:1010E000E9FF64C0EAFF840EEF6E010E836F65C0F6
:1010F000E9FF66C0EAFFEE52080EEF6E65C0E9FF39
:1011000066C0EAFF020EE926000EEA22200EEE6E0D
:10111000040EED6E65C0E9FF66C0EAFF800EEF6E5B
:10112000120000018C6B8D6B020E705D18E165C0C2
:10113000E9FF66C0EAFFEE52080EEF6E65C0E9FFF8
:1011400066C0EAFF020EE926000EEA22280EEE6EC5
:10115000040EED6E65C0E9FF66C0EAFF1DD0745154
:101160000401265D000175510401275904E226C4DB
:1011700074F027C475F02BD96BC0E9FF6CC0EAFF8F
:10118000020EE926000EEA22280EEE6E040EED6E27
:101190006BC0E9FF6CC0EAFFC80EEF6E1200800E54
:1011A0000401205D58E10001C00E736F040123515A
:1011B000030A2FE0010A09E0030A4BE10001EE0EE9
:1011C000716F1D0E726F120E3ED02251F66EF76ACD
:1011D000D890F636F736CE0EF6261E0EF722090008
:1011E000F5CF71F00A00F5CF72F0020E0001F76A38
:1011F0007125F66E7251F7220800F5CF74F0030ED8
:10120000F76A7125F66E7251F7220800F5CF75F076
:101210001200030E225D1AE22251F66EF76AD89090
:10122000F636F736D00EF6261E0EF7220900F5CF59
:1012300071F00A00F5CF72F071C0F6FF72C0F7FFCF
:101240000800F5500001746F756B12000001736B9C
:1012500012000001736B1200D9CFE6FFE1CFD9FF76
:10126000020EE1260401286B296B20511F0B020A94
:1012700011E0030A0CE0010A35E10001738F04015B
:10128000288100017F052EE1040128832BD0000175
:10129000738F28D00001738F040124BF0BD0245119
:1012A0000F0BE96EEA6AD890E936EA36670EE9264E
:1012B000000E0AD024510F0BE96EEA6AD890E93685
:1012C000EA366B0EE926000EEA22EECFDEFFEDCF06
:1012D000DDFFDECFE9FFDDCFEAFFEF50040B02E0D8
:1012E000010E286F000173AF07D0280E716F040E36
:1012F000726F7381020E746F020EE15C02E2E16AAA
:10130000E552E16EE552E7CFD9FF12006D9800017A
:1013100073BF2BD078AF09D0020E706F8D5101E1F1
:1013200000DF00018B6B8A6B120065C0E9FF66C0AD
:10133000EAFFEE52080EEF6E65C0E9FF66C0EAFFF5
:10134000020EE926000EEA22200EEE6E040EED6E6D
:1013500065C0E9FF66C0EAFF8C0EEF6E6BC0E9FF67
:101360006CC0EAFF840EEF6E1200040120AF0DD0B6
:101370000001010E706F8C5101E1D3DE00018B6B17
:101380008A6B895123E140EF08F00001020E706F73
:1013900065C0E9FF66C0EAFFEE52080EEF6E65C059
:1013A000E9FF66C0EAFF020EE926000EEA22200EDF
:1013B000EE6E040EED6E65C0E9FF66C0EAFF840EB6
:1013C000EF6E8B6B8A6B895101E15ADE1200D9CF27
:1013D000E6FFE1CFD9FFE652080EDF6E0001745D33
:1013E000000E75590AE274C0DFFF6F5102E1010E71
:1013F00003D06F0502E1020E6F6FDF500C6AE850F8
:10140000745D746F0C507559756F6BC0E9FF6CC0DB
:10141000EAFFEE52DFCFEFFF280E7D6F040E7E6FE6
:1014200073B118D0DF502DE071C0F6FF72C0F7FF26
:10143000712B000E72230800F550E66E7DC0E9FFA7
:101440007EC0EAFF7D2B000E7E23E552E750EF6E53
:10145000DF06E8D7DF5015E071C0E9FF72C0EAFF90
:10146000712B000E7223EF50E66E7DC0E9FF7EC047
:10147000EAFF7D2B000E7E23E552E750EF6EDF067C
:10148000E9D7E552E552E7CFD9FF1200D9CFE6FF01
:10149000E1CFD9FF020EE12663C0E9FF64C0EAFF95
:1014A000EE52EFCFDFFFDFCF0BF00B500001795D85
:1014B000000E7A5902E279C0DFFFDF500B6E0C6A32
:1014C000E850795D796F0C507A597A6F010EDB6ABA
:1014D000DF50F36E010EDBCFF4FFF350F45C16E245
:1014E000010EDB50EA6A280FE96E040EEA22EF5083
:1014F000E66E76C0E9FF77C0EAFF762B000E772311
:10150000E552E750EF6E010EDB2AE2D7000ED880DD
:101510007955000E7A5527E265C0E9FF66C0EAFFFB
:10152000EE52080EEF6E65C0E9FF66C0EAFF020EDC
:10153000E926000EEA22280EEE6E040EED6E63C060
:10154000E9FF64C0EAFFEF50400B06E165C0E9FF28
:1015500066C0EAFFC80E05D065C0E9FF66C0EAFFB5
:10156000880EEF6E28D065C0E9FF66C0EAFFEE5234
:10157000080EEF6E65C0E9FF66C0EAFF020EE926BD
:10158000000EEA22200EEE6E040EED6E65C0E9FF3D
:1015900066C0EAFF840EEF6E7B517C1107E005D038
:1015A0007CC0FAFF00017B51F96EFADF0001789FE1
:1015B000895101E165DD020EE15C02E2E16AE5527A
:1015C000E16EE552E7CFD9FF1200D9CFE6FFE1CFB8
:1015D000D9FFE6520001738F010EE66EE66AE66AF5
:1015E000710EE66E0F0EE66E20EC10F00B6E050E1F
:1015F000E15E0B50DF6ADF500B6E0C6A080E0B5C6D
:10160000000E0C5810E2DF50040DF3CFE9FFF4CFC9
:10161000EAFF000EE926040EEA22EE6AEE6AEE6A9E
:10162000EE6ADF2AE8D76D8C010EE66EE66AE66A9E
:10163000620EE66E000EE66E20EC10F00B6E050EEC
:10164000E15E0B506D9C0001080E6B6F040E6C6F19
:10165000000E636F040E646F63C065F0666F22C492
:1016600061F0615102E1100E12D0010EE66EE66AE1
:10167000610EE66E000EE66E010EE66EE66A8CEC1A
:101680000EF00B6E060EE15E0B500001200E606F37
:10169000E552E552E7CFD9FF1200D9CFE6FFE1CFFF
:1016A000D9FF020EE126000EDE6E040EDD6EFD0E89
:1016B000DB50E8240D6EFE0EDB50040DF3500D24BC
:1016C000040DF4CF0CF0D9CFE9FFDACFEAFFF350E5
:1016D000EE260C50ED22DECFE9FFDDCFEAFFEF9ED4
:1016E000FD0EDB500AE1FE0EEA6ADB34FE0BEA3641
:1016F000E96E670EE926000E09D0FE0EEA6ADB34B9
:10170000FE0BEA36E96E6B0EE926000EEA22DECF0A
:10171000EEFFDDCFEDFFDECFE9FFDDCFEAFFEF9C8F
:10172000DECFE9FFDDCFEAFF040EE926000EEA2254
:10173000EF8C020EE15C02E2E16AE552E16EE552F5
:10174000E7CFD9FF1200D9CFE6FFE1CFD9FF020ED4
:10175000E126FD0EDBA407D0E66AFE0EDBCFE6FF36
:101760009CDFE552E552FD0EDBA208D0010EE66ECD
:10177000FE0EDBCFE6FF91DFE552E552FE0EDB50B9
:101780000C6A700F0B6E0F0E0C220BC0DEFF0CC02C
:10179000DDFFDECFE9FFDDCFEAFFFD0EDBCFEFFFA0
:1017A000020EE15C02E2E16AE552E16EE552E7CF4A
:1017B000D9FF1200D9CFE6FFE1CFD9FF020EE12613
:1017C000FE0EDB5020E165C0E9FF66C0EAFFEE5285
:1017D000080EEF6E65C0E9FF66C0EAFF020EE9265B
:1017E000000EEA22200EEE6E040EED6E65C0E9FFDB
:1017F00066C0EAFF8C0EEF6E6BC0E9FF6CC0EAFFBB
:10180000840EEF6E3BD0FD0EDB50E8240D6EFE0E15
:10181000DB50040DF3500D24040DF3CF0BF0F4CF87
:101820000CF0000E0B26040E0C220BC0DEFF0CC0C9
:10183000DDFF840EDECFE9FFDDCFEAFFE850EF12D7
:10184000FD0EDB50E8240D6EFE0EDB50040DF35050
:101850000D24010F040DF3CF0BF0F4CF0CF0000EAC
:101860000B26040E0C220BC0DEFF0CC0DDFF840E25
:10187000DECFE9FFDDCFEAFFE850EF12020EE15CB8
:1018800002E2E16AE552E16EE552E7CFD9FF1200CC
:10189000D9CFE6FFE1CFD9FF020EE126FD0EDB50E6
:1018A0000AE0FE0EEA6ADB34FE0BEA36E96E6B0EE6
:1018B000E926000E09D0FE0EEA6ADB34FE0BEA369A
:1018C000E96E670EE926000EEA22EECFDEFFEDCFCD
:1018D000DDFFD9CFE9FFDACFEAFFEE50ED1003E1EB
:1018E000F36AF46A44D0DECFE9FFDDCFEAFF020EEF
:1018F000E926000EEA22FB0EDBCFEEFFFC0EDBCF6B
:10190000EDFFDECFE9FFDDCFEAFFEE52FA0EDBCFCF
:10191000EFFF400EDECFE9FFDDCFEAFFE850EF1624
:10192000880EDECFE9FFDDCFEAFFE850EF12FD0EB3
:10193000DB500AE0FE0EEA6ADB34FE0BEA36E96EA3
:101940006B0EE926000E09D0FE0EEA6ADB34FE0BB0
:10195000EA36E96E670EE926000EEA22EF74DECF62
:101960000BF0DDCF0CF00BC0F3FF0CC0F4FF020E48
:10197000E15C02E2E16AE552E16EE552E7CFD9FFB0
:101980001200D9CFE6FFE1CFD9FF6DA84ED0FE0EF1
:10199000EA6ADB34FE0BEA36E96E6B0EE926000ECE
:1019A000EA22EE50EFCFEAFFE96E400EEE16EE6A45
:1019B000EE6AEE6AFE0EEA6ADB34FE0BEA36E96E88
:1019C0006B0EE926000EEA22EE50EFCFEAFFE96E39
:1019D000EE7CFE0EEA6ADB34FE0BEA36E96E6B0E35
:1019E000E926000EEA22EF74400E0B6EFE0EEA6A44
:1019F000DB34FE0BEA36E96E6B0EE926000EEA22B6
:101A0000EE50EFCFEAFFE96E0B50EF16FE0EEA6ADA
:101A1000DB34FE0BEA36E96E6B0EE926000EEA2295
:101A2000EE50EFCFEAFFE96EEF7CE552E7CFD9FF4A
:021A30001200A2
:0E1A3200DACFE4FFE652E552E5CFDAFF11000D
:101A4000D8CFE4FFE0CFE4FFE46EDACFE4FFE65264
:101A5000E552E5CFDAFFE550E5CFE0FFE5CFD8FF6F
:101A6000100004D8A8EC04F01CD8FCD70F0EC1124B
:101A700002D81CEF04F0FC0E8B1694160001010E28
:101A8000A56F94848250040B01E0010E8E6F82508A
:101A9000040B01E0010E8F6FA06BA16BA26BA36B17
:101AA00012000001A50502E1C7D80CD0A607000E60
:101AB000A75BA85BA95BA651A711A811A91102E118
:101AC000010EA56F200E0001E76E6019E8AE02D08E
:101AD000E73402D0E750605D05E36D50020B01E092
:101AE000120001D812000001A051A11102E1000E64
:101AF00008D0A0C0E9FFA1C0EAFFEF50800B01E0D1
:101B0000010E000946E189D8000927E00401316B84
:101B1000326B0001B651B62B0401336F346B356B59
:101B2000366B376B386B080EE66E310EE66E040EC0
:101B3000E66E010EE66EE66E48EC0CF00B6E050EDE
:101B4000E15E0B50F3CFA0F0F4CFA1F0280E00011E
:101B5000B65D1FE1040EB66F1CD00401316B326B11
:101B6000336B346B356B366B376B386B080EE66E48
:101B7000310EE66E040EE66E010EE66EE66E48EC81
:101B80000CF00B6E050EE15E0B50F3CFA0F0F4CF1E
:101B9000A1F00001A251A31102E1000E08D0A2C0E1
:101BA000E9FFA3C0EAFFEF50800B01E0010E00093E
:101BB00024E1040130A103D08B808B8202D08B9072
:101BC0008B920001A56BE00EA66F220EA76F020E8E
:101BD000A86FA96B010EE66E300EE66E040EE66E7F
:101BE000E66A010EE66E48EC0CF00B6E050EE15E47
:101BF0000B50F3CFA2F0F4CFA3F012008250040BED
:101C000001E0010E00018E5D07E08250040B01E04F
:101C1000010E8E6F82A4010C000C8250040B01E0B7
:101C2000010E00018F5D07E08250040B01E0010E00
:101C30008F6F82A4010C000C0001B751B81104E1B0
:101C4000100EB76F270EB86FB707000EB85B6DA206
:101C500007D0B751B8112EE18B708BB013D027D0BD
:101C60000001605102E18B9022D0600502E18B807F
:101C700009D0020E605D02E18B8019D0040E605D18
:101C800003E18B908B821200100E605D06E1000173
:101C9000B751B8110FE18B700AD0200E605D0AE1D8
:101CA0000001B751B81106E18B708BA002D08B9266
:101CB00012008B82120012001200120012006BEF51
:101CC0000FF012001E0EE66E010EE66EA3EC0BF096
:101CD000E552E552010EE66E300EE66E040EE66E3B
:101CE000E66A010EE66E48EC0CF00B6E050EE15E46
:101CF0000B50F3CFA2F0F4CFA3F012006D840001DB
:101D0000080EAA6F070EAB6FAA07000EAB5BAA51B5
:101D1000AB11FAE16D941200D9CFE6FFE1CFD9FF04
:101D2000FD0EDBCF06F0FE0EDBCF07F0720E0618BD
:101D300001E1075033E0E868061802E17F0E07185A
:101D40002BE0740E061801E1075024E0750E06180A
:101D500001E107501DE0730E061801E1075016E07F
:101D6000030E061801E107500FE0020E061801E10C
:101D7000075008E0010E061801E1075001E010D0FD
:101D8000A1DF0FD09EDF0DD09ADF0BD096DF09D0F8
:101D900092DF07D091DF05D091DF03D0000001D0A2
:101DA00000D0010E00D0E552E7CFD9FF12000001AC
:101DB000280E766F040E776F080E796F7A6BCA0E55
:101DC0007B6F1D0E7C6F788F1200040128A103D059
:101DD0008B808B8202D08B908B920001A56BE00EE2
:0E1DE000A66F220EA76F020EA86FA96B12004D
:021DEE001201E0
:101DF000000200000008D8045500010001020001A3
:101E000009022900010100C0320904000002030197
:101E10000100092111010001223F0007058103088B
:101E20000001070501030800010403090434034D00
:101E3000006900630072006F006300680069007051
:101E400000200054006500630068006E006F006CA5
:101E5000006F0067007900200049006E0063002ECB
:101E6000002E034B006500790062006F0061007274
:101E70000064002000440065006D006F0000000059
:101E8000000000000000000000000000000000054D
:101E9000010906A101050719E029E71500250175CB
:101EA0000195088102950175088103950575010565
:101EB000081901290591029501750391039506758D
:101EC00008150025650507190029658100C0001E59
:061ED000291E2D1E611EFB
:0A1ED600040120511F0B010801E078
:101EE0001200245101E01200060E215D1EE1235173
:101EF000230A1BE0010A0CE0030A17E10001610557
:101F000014E10001120E716F1E0E726F090E09D0DE
:101F1000000161050AE100018F0E716F1E0E726FE4
:101F20003F0E746F756BC00E736F04012051600B10
:101F3000E842E842E842E842E842010801E01200D3
:101F400021510B0A28E0080A1BE0090A13E0080ADD
:101F500007E00B0A03E0080A23E01200D7EF0EF0B7
:101F60000001B90E716F000E726F010E746F756B08
:101F7000C10E0FD00001800E736F23C4B9F01200A0
:101F80000001BA0E716F000E726F010E746F756BE7
:101F9000810E736F12000001800E736F22C4BAF0BD
:021FA00012002D
:0E1FA2002A0EF66E080EF76E000EF86E0001A5
:101FB0000900F550B16F0900F550B26F03E1B16748
:101FC00001D03DD00900F550AC6F0900F550AD6F60
:101FD0000900F550AE6F09000900F550E96E0900DF
:101FE000F550EA6E090009000900F550AF6F0900CD
:101FF000F550B06F09000900F6CFB3F0F7CFB4F099
:10200000F8CFB5F0ACC0F6FFADC0F7FFAEC0F8FF3B
:102010000001AF5302E1B05307E00900F550EE6E46
:10202000AF07F8E2B007F9D7B3C0F6FFB4C0F7FFC7
:10203000B5C0F8FF0001B107000EB25BBFD71200B8
:10204000FE0EE3CFE9FFFF0EE3CFEAFFE9CFF3FF98
:10205000EACFF4FFFB0EE35003E1FC0EE35009E08E
:10206000FB0EE30602E2FC0EE306FD0EE350EE6E0D
:04207000F1D7120092
:0C207400000EF36E00EE00F0040E01D828
:102080001200EA6002D0EE6AFCD7F350E960120059
:04209000EE6AFCD721
:0C20940013EE00F023EE00F0F86A0A9C46
:1020A000D1EC0FF058EC10F031EC0DF0FBD7120032
:0220B00012001C
:0320B20004000027
:00000001FF
